:020000040000FA
:1000000000308B0000308500003086008316C5303C
:1000100081001E308500F030860083129601900129
:100020009A0103101A14950106148615061A151460
:10003000861A9514061B1515861B95150610861134
:100040006F209220F32034202D2034202D203420C6
:100050002D2034202D202D2020285F3093000000FB
:100060000000930B2F28080003308A00100800239B
:100070008A019700083094000510970D6920031C31
:100080000514632005146920940B3C280510692091
:10009000961E051463200514692005106920961E1C
:1000A0000514632005146920110897000830940096
:1000B0000510970D6920031C0514632005146920A1
:1000C000940B58280800083093000000930B652813
:1000D0000800023093000000930B6B280800980181
:1000E0000430990086010314860D0310061A902827
:1000F000980A861A9028980A061B9028980A861B48
:100100009028980A85189028980A05199028980A26
:1001100085199028980A051A9028980A990B74282E
:10012000860108009A1EE428981AEC289A01031008
:100130001A14043018020318A0280130F620DE2813
:10014000083018020318A9280230F620043098025B
:10015000DE280C3018020318B2280130F6200430D3
:100160009802DE28103018020318BB280230F6204F
:1001700008309802DE28143018020318C42803300F
:10018000F62010309802DE28183018020318CD2807
:100190000430F62014309802DE281C3018020318B0
:1001A000D6280330F62014309802DE2820301802BA
:1001B0000318DE280430F6201830980202308A0036
:1001C000180800228A0191001A18EF289A18EF28BF
:1001D000111091109A0D080091019001080011145E
:1001E00091149A0D0800851CF328080089008316D5
:0E01F0000814831208089000150890070800F4
:10040000820700340C3430343C34C034CC34F03403
:04041000FC34003484
:100600008207AA34C03480343034F034B03420341B
:10061000E034A0340C34CC348C343C34FC34BC3462
:100620002C34EC34AC340834C83488343834F834DE
:10063000B8342834E834A8340334C334833433342E
:10064000F334B3342334E334A3340F34CF348F344E
:100650003F34FF34BF342F34EF34AF340B34CB345A
:100660008B343B34FB34BB342B34EB34AB340234AB
:10067000C23482343234F234B2342234E234A2341A
:100680000E34CE348E343E34FE34BE342E34EE344A
:10069000AE340A34CA348A343A34FA34BA342A3496
:1006A000EA34003440346034973470344834683469
:1006B0005834783444346434543474344C346C34A2
:1006C0005C347C3442346234523472344A346A3496
:1006D0005A347A3446346634563476344E346E3472
:0206E0005E3486
:02400E00F93F78
:104200000200140028003C00000000000000000034
:10421000000000000000000000000000000000009E
:10422000000000000000000000000000000000008E
:10423000000000000000000000000000000000007E
:10424000000000000000000000000000000000006E
:10425000000000000000000000000000000000005E
:10426000000000000000000000000000000000004E
:10427000000000000000000000000000000000003E
:00000001FF
